:100000008B01813062001A288B10A800030EA90012
:10001000241186182415A40CA30CAA16A20B1528CB
:100020000B30A200BB152308A500290E8300A80EE3
:10003000280E0900FF309F0085018601FF30650012
:10004000660020308400423C8001840AFF3E031D8C
:100050002428863084001830AB000B30A20000301A
:10006000AB210F3065006430AB21013062000030FD
:10007000AB210030AB210030AB210030AB21003090
:10008000AB210030AB210030AB210030AB21003080
:10009000AB210030AB21001080143230AB21F330A3
:1000A0007021C8307021F330702164307021F3303A
:1000B000702150307021F23070219A21033C0319D5
:1000C0003B17E830702103307021E6307021F330A7
:1000D0007021C8307021F43070216021E930702126
:1000E00003180028FA3C031D00289A210318002851
:1000F0006039203C031D00283B1A89289A210318E7
:100100008728BB1A89289A210318882889283B1632
:10011000BB160330A1003B1BA10AAE010008060676
:10012000043903199828BB130F306500FF30800095
:100130008B170B16BB1DB028BB112E083C3E84004C
:100140002508800086308400AE0AA10BFB2803300E
:10015000A1003B1BA10AAE013B141830AB00FB28E9
:100160003B1CCB283B10BB14B10101303C1AFF30C3
:10017000BD08031DB1003D083C1A003C2F070318C1
:10018000FF30AF00B300B307031CB307031CFB2809
:10019000FF30B300FB28BB1CE628BB103B15B201A7
:1001A0000130BC1AFF30BE08031DB2003E08BC1A65
:1001B000003C30070318FF30B000B500B507031C42
:1001C000B507031CFB28FF30B500FB283B1DFB28AF
:1001D0003B113C0DAD00AD0D2D091C39AD001C3C93
:1001E000031D6021BB1FF8280008E3392D0480009F
:1001F0003F083B1BC007811F9A282A3081026400F8
:10020000AC0B1429AB0B14291830AB000B122108CE
:100210003B1BFF3E033C031D132922080B3C031D1F
:10022000132906186E280B163308B407031C23295C
:10023000AF0803192329AF033108B702370C01397E
:1002400037060339B9003508B607031C3229B00850
:1002500003193229B0033208B807380C01393806BF
:100260000339BA00861A39290230C10000178017F5
:10027000C001C00803194D290130C01F003CC00750
:10028000C107410C01394106AD0000083F392D1866
:100290004038AD188038BB1B80000310390D39077A
:1002A00039073A04BB1B6500AA0B9A280B12AA084F
:1002B000031D5E290B30A200AA1689280B169A2866
:1002C000BB1B080005090F390319061D0800BB17E1
:1002D0000330B900BA000230B700B800C10008000E
:1002E0008B01AD00A600A701A70900106430B4215E
:1002F0000830A0000130AD0C0318A706A00B7B2925
:100300000B30A0000014801064000001013E0319AE
:10031000002806188629A70CA60C031C80100318B9
:1003200080140001013E03190028061C9229A00B2D
:1003300084298B018B170B162830A00064006430D1
:10034000B421BB1DA729BB11250803100800A00B71
:100350009E2903140800A0006400F930FF3E031D2D
:10036000AE29A00BAC290800FF3E031DB4290800EC
:00000001FF
